:0200000480007A
:100000006F00C0006F20802C6F20402C93000000F8
:10001000130100009301000013020000930200008E
:100020001303000093030000130400009304000076
:10003000130500009305000013060000930600005E
:100040001307000093070000130800009308000046
:100050001309000093090000130A0000930A00002E
:10006000130B0000930B0000130C0000930C000016
:10007000130D0000930D0000130E0000930E0000FE
:10008000130F0000930F000097020000938202F804
:1000900073905230179100001301C1E4F32240F134
:1000A0009392C2003301510073100134EF20900B82
:1000B000173500001305858B6F20006B8332851088
:1000C000739012148330850003310501833185015B
:1000D000033205028332850203330503833385032C
:1000E000033405048334850483358505033605060A
:1000F00083368506033705078337850703380508E8
:10010000833885080339050983398509033A050AC7
:10011000833A850A033B050B833B850B033C050CA7
:10012000833C850C033D050D833D850D033E050E87
:10013000833E850E033F050F833F850F033505057D
:10014000730020107311011423341100233C31007B
:10015000233041022334510223386102233C7102CF
:1001600023308104233491042338A104233CB104B7
:100170002330C1062334D1062338E106233CF1069F
:10018000233001092334110923382109233C310983
:100190002330410B2334510B2338610B233C710B6B
:1001A0002330810D2334910D2338A10D233CB10D53
:1001B0002330C10F2334D10F2338E10F233CF10F3B
:1001C000F312011423385100F32200102330511090
:1001D000F322101423345110F32230142338511019
:1001E000F3222014233C5110130501006F208033AB
:1010000000000000000000000000000000000000E0
:1010100000000000000000000000000000000000D0
:1010200000000000000000000000000000000000C0
:1010300000000000000000000000000000000000B0
:081040000000000000000000A8
:10200000B367B500B3E7C70093F77700B306C50021
:10201000638407023386C50093070500637ED502FB
:1020200003C705009385150093871700A38FE7FE6C
:10203000E398C5FE67800000E37ED5FE93070500A8
:1020400003B70500938787009385850023BCE7FECF
:10205000E3E8D7FE6780000067800000130101FFFE
:10206000B367C500233081002334110093F7770054
:10207000130405003307C500638207026376E50099
:1020800093F5F50FEFF09FFD8330810013050400F9
:1020900003340100130101016780000093F5F50F7F
:1020A00093968500B3E6B60093970601B3E7D70091
:1020B00093960702B3E6F600E378E5FC9307050084
:1020C0009387870023BCD7FEE3ECE7FE83308100D3
:1020D00013050400033401001301010167800000AF
:1020E00083470500638E07009307050003C71700A9
:1020F00093871700E31C07FE3385A7406780000025
:1021000013050000678000008347050093851500D4
:102110001305150003C7F5FF638A0700E386E7FE92
:102120001B8507003B05E5406780000013050000A4
:102130006FF05FFFB367B50093F77700639E070208
:10214000137886FF330805016378050393070500BC
:102150006F000001938787009385850063F807016E
:1021600083B6070003B70500E386E6FE3385A74084
:102170003306A640138507003386C5006F00400173
:1021800003C705008347F5FF93851500639AE700B1
:1021900013051500E396C5FE1305000067800000D7
:1021A0003B85E740678000009307050003C70500F3
:1021B0009387170093851500A38FE7FEE31807FEAA
:1021C000678000000347050093060002930705009F
:1021D0006318D70003C7170093871700E30CD7FED7
:1021E0009306D0026300D7069306B0026300D704BB
:1021F00083C60700930500006382060413050000F0
:1022000093871700131725001B8606FD83C607005A
:102210003307A700131717003305E600E39206FE05
:10222000638005023305A0406780000083C6170065
:102230009305000093871700E39206FC1305000046
:102240006780000083C6170093051000938717006E
:10225000E39606FA130500006FF09FFE8347050022
:10226000638007049305101017F7FFFF130787D942
:10227000939505030336070013051500B3E6B70071
:10228000630A060097F7FFFF23BE07DA83370700CC
:10229000E39A07FE2330D70083470500E39C07FC41
:1022A0006780000017F7FFFF1307C7D583370700C4
:1022B000638A070097F7FFFF23B607D88337070025
:1022C000E39A07FE2330A7006F000000130101FF0F
:1022D0001305903423341100EFF0DFFC130101FEED
:1022E0001306810093077101130890006F008000AE
:1022F000930707009376F500138706009305000304
:102300006374D800930570053B07B7002380E7008E
:10231000135545001387F7FFE31CF6FC8347810044
:10232000230C0100638207041305101093060600B6
:1023300017F7FFFF130707CD1315050383350700B4
:102340009386160033E6A700638A050097F7FFFF20
:1023500023BA07CE83370700E39A07FE83C7060038
:102360002330C700E39C07FC1301010267800000D3
:10237000130101FF37F8FFFF233411003307050174
:10238000B7E703006378F7141357C5009306076097
:1023900017260000130606C793973600B307F6000A
:1023A00083B70700337505016390070E976500003A
:1023B0009385C5C503B805006302081483378800F8
:1023C0009768000083B808C423B0F500638E170F28
:1023D0008337080093983600B308160193D7C700D7
:1023E0009397A70013E3F70D93E5F70123B0680077
:1023F00073000512971700009387C7C01317470093
:10240000B387E70003B7070063140710033708001A
:10241000B708040023B0E7000337880023B4E700BF
:10242000F3A80810B707E0FFB307F500371800005E
:10243000130705003388070103BF070083BE870029
:1024400003BE070103B387012330E7012334D7011B
:102450002338C701233C670093870702130707024D
:10246000E39C07FD7390081093973600B306F600BF
:1024700023B0B600730005120F10000083308100F6
:10248000130101016780000013F70704630A0702C4
:1024900013F70708631A07041307F00093E7070808
:1024A0006394E50493963600B306D60023B0F60095
:1024B0007300051283308100130101016780000061
:1024C00093E707046FF01FFE9767000023BC07B275
:1024D0006FF01FF0171500001305C582EFF01FD82D
:1024E00013053000EFF01FDC1715000013050586FB
:1024F000EFF0DFD613053000EFF0DFDA171500003C
:1025000013054589EFF09FD513053000EFF09FD9F3
:102510001715000013058589EFF05FD4130530000F
:10252000EFF05FD883358511130101F82338810658
:10253000233C11062334910623302107233C310527
:10254000233841052334510523306105233C7103B1
:1025500023388103233491032330A103233CB101A9
:102560009307800013040500638AF50E930720008B
:102570006380F506938745FF130710006376F70025
:102580009307F0006392F51A03350411EFF05FDE54
:102590001305040003340107833081078334810667
:1025A0000339010683398105033A0105833A810421
:1025B000033B0104833B8103033C0103833C810211
:1025C000033D0102833D8101130101086FD01FAF5C
:1025D000033785109377370063980706EF0780006D
:1025E000731030000327070083A70700630AF7046E
:1025F0001305101093071004970600009386067FBA
:1026000017F7FFFF130707A013150503833507000E
:102610009386160033E6A700638A050097F7FFFF4D
:1026200023B207A283370700E39A07FE83C7060099
:102630002330C700E39C07FC13053000EFF09FC672
:1026400013051000EFF01FC61715000013050584D1
:10265000EFF0DFC013053000EFF0DFC403290505FC
:10266000371C0000971400009384C499972B000036
:10267000938B4B99370B0400B70AE0FF976D00006E
:10268000938D4D98176A0000130A4A98B7F9030012
:102690006F0080012334F70023B0FD00B71700005E
:1026A000330CFC00630E3C0B9357CC001394470093
:1026B0003387840003370700E30207FE9387076030
:1026C00093973700B387FB0083BC070093F70C0494
:1026D000638E0706732D0B1037160000B3055C01DF
:1026E00013050C002334B100EFF0DFA4630E0500E6
:1026F00093FC0C088335810063800C0437160000BE
:1027000013050C00EFF0DF8FB387840073100D10FA
:1027100003B70D0023B00700E31E07F623B0FD004A
:102720002330FA006FF09FF7170500001305857836
:10273000EFF0DFB26FF05FF0170500001305857151
:10274000EFF0DFB113053000EFF0DFB51705000043
:102750001305C56CEFF09FB013053000EFF09FB488
:1027600013050900EFF01FB4F32740F1639A07182F
:102770009747000093870789130101ED93D7C7009E
:1027800023308112175800001308C887130405006E
:102790009397A700173500001305C586233411123F
:1027A0009356C5001357C80093E7170097280000F9
:1027B000938848851306F0FF233CF5FE9396A60008
:1027C0001317A700B707002093E61600136717003A
:1027D00093D5C8001313F6039387F70C233CF8FE38
:1027E00023B0D8002330E500B3E7650073900718E5
:1027F00073270018639EE7141356B6009307F00181
:102800009702000093824201F39252307310063B0C
:102810007390073A739052301308F0BF13185801A1
:1028200097E7FFFF93874792B3870701739057108D
:10283000F3270034B387070173900714B7B700007C
:102840009B87071073902730B7E701009B870760CD
:10285000739007307350403017170000130787B983
:102860009307083EB3060701B307F700B70808004F
:1028700017560000233CD67817130000130383F685
:102880009756000023B0F6789388F80393078000EA
:102890001308080113D61700B3861701B347F600D3
:1028A000B30507019396C600939757002330D700CE
:1028B0002334B70093F7070213070701B367F60045
:1028C000E31AE3FC13060012930500001305010050
:1028D0009717000023B407F0EFF04FF8B707008018
:1028E0003304F4001305010023348110EFD00FFDF1
:1028F0008330811203340112130101136780000039
:1029000013071000B7E78F0E37060800938747CAF2
:102910001306C6FF1315F7019316E7036F00C001F6
:102920002F20070013D71700B3C7E7009397E703DB
:10293000B3F7D700B3E7E70033F7C70093F5170005
:102940003307A700E39E05FC032007006FF09FFDFF
:102950001705000013050559EFF05F9013053000CF
:10296000EFF05F9467800000B70000801BD7004045
:10297000B70300809301200063147736B70000800E
:102980001BD71040B70300C093013000631A77349F
:10299000B70000801BD77040B70300FF93014000D1
:1029A00063107734B70000801BD7E040B703FEFF09
:1029B0009301500063167732B70000809B801000AF
:1029C0001BD7F0419303F0FF93016000631A773047
:1029D000B70000809B80F0FF1BD70040B70300804A
:1029E0009B83F3FF93017000631C772EB700008078
:1029F0009B80F0FF1BD71040B70300409B83F3FF81
:102A000093018000631E772CB70000809B80F0FF4D
:102A10001BD77040B70300019B83F3FF9301900025
:102A20006310772CB70000809B80F0FF1BD7E0403D
:102A3000B70302009B83F3FF9301A0006312772A80
:102A4000B70000809B80F0FF1BD7F041930300008C
:102A50009301B00063167728B78081819B8010189E
:102A60001BD70040B78381819B8313189301C0005B
:102A700063187726B78081819B8010181BD7104080
:102A8000B7C3C0C09B83030C9301D000631A7724A3
:102A9000B78081819B8010181BD77040B70303FF5C
:102AA0009B8333309301E000631C7722B7808181E0
:102AB0009B8010181BD7E040B703FEFF9B83636029
:102AC0009301F000631E7720B78081819B801018EE
:102AD0001BD7F0419303F0FF9301000163127720AD
:102AE000B720F1FF9B8050349390C00093808067A3
:102AF0001BD70040B75334129B8383679301C002F6
:102B00006310771EB720F1FF9B8050349390C00074
:102B1000938080671BD74040B74323019B83735644
:102B20009301D002631E771AB72009009B805034AE
:102B30009390C000938080671BD70040B7533492B6
:102B40009B8383679301E002631C7718B720090019
:102B50009B8050349390C000938080671BD7404087
:102B6000B74323F99B8373569301F002631A7716D8
:102B7000B70000809BD07040B70300FF93011001A5
:102B80006390701613020000B70000801BD77040DE
:102B9000130307001302120093022000E31652FEF3
:102BA000B70300FF93012001631C7312130200009E
:102BB000B70000801BD7E04013000000130307009C
:102BC0001302120093022000E31452FEB703FEFF2B
:102BD000930130016316731013020000B7000080E8
:102BE0009B8010001BD7F041130000001300000071
:102BF000130307001302120093022000E31052FE99
:102C00009303F0FF93014001631C730C1302000057
:102C1000B70000801BD770401302120093022000FF
:102C2000E31852FEB70300FF93015001631A770ABD
:102C300013020000B7000080130000001BD7E04023
:102C40001302120093022000E31652FEB703FEFFA8
:102C5000930160016316770813020000B70000803B
:102C60009B80100013000000130000001BD7F041F0
:102C70001302120093022000E31252FE9303F0FFAE
:102C800093017001631E77049B50F0419303000091
:102C900093018001639670049300F0011BD0C04142
:102CA0009303000093019001631C70029B0070006D
:102CB000939050031BD7C041930300009301A001E0
:102CC000631077029B00F0009390C0011BD7404037
:102CD000B70300FF9301B00163147700631A30005B
:102CE00013951100630005001365150073000000C3
:0C2CF0001305100073000000731000C0FA
:102D0000417373657274696F6E206661696C656486
:102D10003A2061646472203E3D202831554C203CAD
:102D20003C203132292026262061646472203C2018
:102D30003633202A202831554C203C3C2031322982
:102D40000A00000000000000417373657274696F2F
:102D50006E206661696C65643A20212870745B336B
:102D60005D5B616464722F2831554C203C3C2031FE
:102D700032295D2026203078303830292026262040
:102D80006361757365203D3D203078660A00000060
:102D9000417373657274696F6E206661696C6564F6
:102DA0003A206E6F64650A00417373657274696FCF
:102DB0006E206661696C65643A20757365725F6D3B
:102DC000617070696E675B616464722F2831554C65
:102DD000203C3C203132295D2E61646472203D3DEF
:102DE00020300A0000000000417373657274696F3F
:102DF0006E206661696C65643A202122696C6C659D
:102E000067616C20696E737472756374696F6E228A
:102E10000A00000000000000417373657274696F5E
:102E20006E206661696C65643A2070745B335D5B2B
:102E3000616464722F2831554C203C3C203132298A
:102E40005D20262030783034300A00000000000079
:102E5000417373657274696F6E206661696C656435
:102E60003A2070745B335D5B616464722F28315566
:102E70004C203C3C203132295D20262030783038EF
:102E8000300A000000000000417373657274696FBE
:102E90006E206661696C65643A2074662D3E6570CB
:102EA0006320252034203D3D20300A000000000032
:102EB000417373657274696F6E206661696C6564D5
:102EC0003A202122756E65787065637465642065AB
:102ED0007863657074696F6E220A0000000000005C
:102EE000417373657274696F6E206661696C6564A5
:102EF0003A202122756E737570706F72746564204C
:0C2F000073617470206D6F6465220A001C
:040000058000000077
:00000001FF
